:100000000C941E060C94C1270C94EE270C94460603
:100010000C9446060C94E9120C9446060C94460681
:100020000C9446060C9446060C9446060C94460620
:100030000C9446060C9446060C9446060C94460610
:100040000C941B280C9446060C94092C0C944C2CF4
:100050000C9446060C9446060C9446060C944606F0
:100060000C9446060C9446065218B4189318961829
:1000700099189C189F18A218A518B418AE18E6195C
:10008000E819E819E619E819E819E819E819E8196A
:10009000E819E819E819E819E819E819E819E81958
:1000A0006C19E819E819E819E819E819DD18E819D0
:1000B000E819E819E819E819E819E819E819E81938
:1000C000E819E819E819E819E819E8197819781908
:1000D0007819781978197819781978197819E81928
:1000E000E819E819E819E819E819DD1877197719F6
:1000F00077197719E81985198B19911997199D198D
:10010000A319A919AF19B919C319CD19D7191E19EE
:10011000E018E819E819E819E8196C19E819E8195C
:10012000E819E819E819E819E819E81976197619AB
:1001300076197619E81985198B19911997199D194E
:10014000A319A919AF19B919C319CD19D7191E19AE
:10015000E018E819E819E819E8196C191B1A1B1AB4
:100160001B1A1B1A1B1A1B1A1B1A1B1A1B1A1B1AE7
:100170001B1A1B1A1B1A311B311B311B311B311B64
:10018000311B601A6A1A741A7E1ADB1AE51AF41AFD
:10019000051B8D1CA21CAE1CB71CC61CEB1CF41C42
:1001A0003D1D061D502056205C20632071209320A9
:1001B000B120456E746572206D656E752E2E2E0011
:1001C000546F67676C6564206D6963726F50504D42
:1001D00000546F67676C656420696E76657274653C
:1001E000642050504D2100546F67676C6564205443
:1001F00058206D7574696E672100546F67676C6570
:10020000642074656C656D65747279210050726F3D
:10021000746F636F6C206572726F72207769746897
:100220002052580054696D656F7574207768656E4B
:1002300020636F6E6E656374696E6720746F205201
:100240005800507265737320616E79206B65792058
:10025000746F2063616E63656C00436F6E6E6563DF
:1002600074696E6720746F2052582C20706F776508
:100270007220757020746865205258202877697440
:10028000682062696E6420706C7567206966206EF4
:100290006F74207573696E6720616C776179732064
:1002A00062696E642900546F67676C656420276912
:1002B0006D6D656469617465206F75747075742700
:1002C00000546F67676C65642027736C61766520E6
:1002D0006D6F64652700546F67676C6564202761E4
:1002E0006C776179732062696E642700546F676769
:1002F0006C65642050504D206368616E6E656C20A3
:100300006C696D69740053657420525353492069B8
:100310006E6A656374696F6E206368616E6E656C8A
:100320002028303D3D64697361626C652900536526
:10033000742050504D206D696E696D756D20737914
:100340006E630053657420626561636F6E20696E31
:1003500074657276616C0053657420626561636FC9
:100360006E2064656C617900536574206265616319
:100370006F6E206672657175656E637920696E2097
:10038000487A3A20303D64697361626C652C205074
:10039000783D504D52206368616E6E656C20782CFC
:1003A0002046783D465253206368616E6E656C202E
:1003B00078005365742050574D2073746F7020641B
:1003C000656C61792028302064697361626C6564B2
:1003D0002C20312D323535203D3D20302E317320FB
:1003E0002D2035306D696E29005365742050504DB5
:1003F0002073746F702064656C61792028302064EC
:10040000697361626C65642C20312D323535203D75
:100410003D20302E3173202D2035306D696E29003E
:10042000536574206661696C736166652064656CF0
:1004300061792028302064697361626C65642C20C6
:10044000312D323535203D3D20302E3173202D2089
:1004500035306D696E29002A2A2A2A2A2A2A2A2A50
:100460002A2A2A2A2A2A2A2A2A2A2A2A2A2A2A2AEC
:100470002A2A2A2A0052582041636B6564202D20C5
:1004800072657665727420737563636573736675E0
:100490006C21002A2A2A2A2A2A2A2A2A2A2A2A2AAD
:1004A0002A2A2A2A2A2A2A2A2A2A2A2A2A2A2A2AAC
:1004B000002A2A2A2A2A2A2A2A2A2A2A2A2A2A2AC6
:1004C0002A2A2A2A2A2A2A2A2A2A2A2A2A2A00528E
:1004D000582041636B6564202D20757064617465DC
:1004E000207375636365737366756C21002A2A2A0D
:1004F0002A2A2A2A2A2A2A2A2A2A2A2A2A2A2A2A5C
:100500002A2A2A2A2A2A2A2A2A2A0056616C696457
:100510002063686F69636573206172653A205B319F
:100520005D2D5B31365D20286368616E6E656C20E1
:10053000312D31362900536574206F7574707574D0
:1005400020666F7220706F727420005B585D2061AE
:10055000626F7274206368616E67657320616E6498
:10056000206578697420525820636F6E6669670051
:100570005B535D20736176652073657474696E6783
:100580007320746F205258005B525D20726576654F
:1005900072742052582073657474696E6773207486
:1005A0006F2064656661756C747300557365206EA9
:1005B000756D62657273205B312D445D20746F2010
:1005C0006564697420706F727473205B452D515D92
:1005D00020666F722073657474696E677300202DD6
:1005E00020726563656976657220636F6E66696700
:1005F000757261746F722C20727820737720000AF4
:100600000A6F70656E4C52536E67200053657420FC
:1006100073657269616C2062617564726174653AB8
:10062000200056616C69642063686F696365733A82
:100630002031202D20342B34202F2032202D203823
:10064000202F2033202D20382B34202F2034202D14
:10065000203132202F2035202D2031322B34202FF5
:100660002036202D20313600536574204368616E9A
:100670006E656C20636F6E6669673A20005365741F
:100680002044617461726174652028302D32293AEA
:10069000200053657420486F70206368616E6E653A
:1006A0006C7320286D61782032342C207365706162
:1006B000726174656420627920636F6D6D61732966
:1006C0002076616C69642076616C75657320312DCC
:1006D0003235353A2000536574206368616E6E656B
:1006E0006C2073706163696E6720287831306B48C5
:1006F0007A293A200053657420524620706F77653E
:10070000722028302D37293A200053657420524634
:10071000206D6167696320286865782920652E67E8
:100720002E20307844454144463030443A2000532E
:1007300065742062617365206672657175656E63AC
:10074000792028696E20487A293A20005B5A5D207A
:10075000656E746572207265636569766572206383
:100760006F6E66696775726174696F6E2075746902
:100770006C79005B465D20646973706C61792061FF
:10078000637475616C206672657175656E63696509
:10079000732075736564005B525D2063616C6375E3
:1007A0006C6174652072616E646F6D206B65792079
:1007B000616E6420686F70206C697374005B495DC2
:1007C000207265696E697469616C697A6520736508
:1007D0007474696E677320746F20736B65746368DB
:1007E0002064656661756C7473005B585D2072658A
:1007F00076657274206368616E67657320616E64EC
:100800002065786974206D656E75005B535D20739B
:100810006176652073657474696E677320746F20E8
:10082000454550524F4D20616E64206578697420B3
:100830006D656E7500557365206E756D62657273BA
:10084000205B302D395D20746F20656469742070E1
:100850006172616D657465727300202D2053797328
:1008600074656D20636F6E66696775726174696F18
:100870006E000A0A6F70656E4C52536E672000510D
:1008800029204F7574707574206265666F726520DB
:100890006C696E6B20283D465329203A2000502970
:1008A00020536C617665206D6F64652028657870D3
:1008B0006572696D656E74616C293A20004F29205C
:1008C00054696D65642042494E44206174207374FC
:1008D000617274757020203A20004E292050504DCE
:1008E000206F7574707574206C696D69746564200F
:1008F000202020203A200044495341424C454400E6
:100900004D292050504D205253534920746F20637D
:1009100068616E6E656C202020203A20004C2920F2
:1009200050504D206D696E696D756D2073796E63E1
:10093000202875732920203A200044495341424C15
:100940004544004B29204661696C736166652062ED
:100950006561636F6E20696E74762E2028312D32AA
:10096000353573293A20004A29204661696C736144
:10097000666520626561636F6E2064656C617920D5
:1009800028302D323535203D3E20313073202D204A
:100990003135306D696E293A200049292046616958
:1009A0006C7361666520626561636F6E206672714B
:1009B0002E203A200048292050574D2073746F7024
:1009C0002064656C6179202020202020203A2000BE
:1009D00047292050504D2073746F702064656C61FE
:1009E00079202020202020203A200046292046611E
:1009F000696C736166652064656C617920202020D4
:100A00002020203A200050574D206368616E6E65AB
:100A10006C200066756E6374696F6E3A2000292041
:100A2000706F72742000506F776572546F776572C3
:100A300000445446205548462033322D62697420C4
:100A400031306368004F70656E4C52536E67525878
:100A5000206D696E6920342F36636800466C7974A6
:100A6000726F6E2F4F72616E6765525820554846FF
:100A70002038636800525820747970653A20004429
:100A8000697361626C656400487A00203D3D200016
:100A900043616C63756C61746564207061636B6540
:100AA0007420696E74657276616C3A200042292068
:100AB0004D6963726F202868616C66292050504D23
:100AC000202020203A00412920496E766572746505
:100AD000642050504D20696E20202020203A0030A4
:100AE00029204D7574652062757A7A657220286DAB
:100AF0006F73746C79293A003929205365726961E2
:100B00006C2062617564726174653A00736D617224
:100B100074506F7274004672536B79005472616E38
:100B200073706172656E740044697361626C6564B0
:100B30000038292054656C656D657472793A2020FF
:100B40002020202020003729204368616E6E656CCC
:100B500020636F6E6669673A202000362920446161
:100B60007461726174652028302D32293A2020206A
:100B700000352920486F70206368616E6E656C7364
:100B80003A2020202020003429204368616E6E65C1
:100B90006C2073706163696E673A202000332920EE
:100BA000524620706F7765722028302D37293A2001
:100BB0002020003229205246206D616769633A2067
:100BC0002020202020202020003129204261736530
:100BD000206672657175656E63793A202020000089
:100BE00000000700020100000304060000000000EE
:100BF00000000001020408102040800102040810D7
:100C00002001020408102004040404040404040263
:100C10000202020202030303030303000000002395
:100C2000002600290000000000250028002B0000FD
:100C3000000000240027002A00003A2D11241FBEC6
:100C4000CFEFD8E0DEBFCDBF13E0A0E0B1E0E2E837
:100C5000F0E602C005900D92A83CB107D9F716E066
:100C6000A8ECB3E001C01D92AC38B107E1F71CE07D
:100C7000CCE3DCE004C02297FE010E94432ECA337D
:100C8000D107C9F70E94762D0C943F300C940000D8
:100C900080917105813019F482E080937105809113
:100CA0007105833019F484E0809371050895A89547
:100CB0000895DC01ED91FC910190F081E02D099502
:100CC00008952091720530917305382748E0C901D5
:100CD000880F991F37FF06C09C0151E2252750E17C
:100CE000352701C09C01415091F730937305209343
:100CF0007205089588E38093740580E092ECA1E08A
:100D0000B0E08093750590937605A0937705B09336
:100D1000780587E08093810580E091EAACEBB3E34E
:100D20008093790590937A05A0937B05B0937C0519
:100D300085E0809382058DEE9EEFADEABEED809357
:100D40007D0590937E05A0937F05B0938005E3E831
:100D5000F5E080E090E0863028F4DC01AE54BC4F32
:100D60002C9101C020E0219301968831910599F7DB
:100D700082E080939B058AE080939C05089580E043
:100D80009EECADEEB4E38093B9059093BA05A093C1
:100D9000BB05B093BC0580E090E0A0E0B0E5809397
:100DA000BD059093BE05A093BF05B093C005E1ECCF
:100DB000F5E080E081938F5F8031E1F70895A0E056
:100DC000B0E0E5EEF6E00C940C2ED82F0E947128CE
:100DD0006115710581059105C9F30E94AF2E10922E
:100DE0007D0510927E0510927F0510928005C4E06B
:100DF000812C912C54018A94C0907D05D0907E0561
:100E0000E0907F05F0908005FE2CED2CDC2CCC24AE
:100E10000E94AA2EA50194010E94EB2D6C0D7D1D50
:100E20008E1D9F1D60937D0570937E0580937F05C9
:100E300090938005C15001F7DD2309F450C003E809
:100E400015E0E801A12CB12C62E3C62ED12CE12CD7
:100E5000F12C8881882309F442C0B39419F40E94CC
:100E60007A063DC00E94AA2EA70196010E94EB2D92
:100E7000E1E0E60FA3E8B5E08A2F801B8A1520F495
:100E80008D918E13F9CFE9CF2091820530E0A0E15A
:100E9000B7E20E94832D9B01AC01AE2FB0E00E940F
:100EA000922D4090790550907A0560907B05709066
:100EB0007C05640D751D861D971D4090B9055090E9
:100EC000BA056090BB057090BC05461657066806CB
:100ED000790618F2E993A39488E1A812BACFCDB7A6
:100EE000DEB7E0E10C94282E8436910520F4BC0195
:100EF00080E090E017C09C018E3B910528F42A55B4
:100F00003109AAE0B0E00CC0823D910528F4245BD1
:100F10003109A4E6B0E004C02D5C3109A8E5B2E0D7
:100F20000E94832DA4E6B0E09B01AC010E94922DAB
:100F3000089590E08C599F4F0E947407089561E0D6
:100F40008AE00E941E2960E08AE00E9457290895E5
:100F5000892B11F061E001C060E08AE00E9457290E
:100F6000089560E089E00E941E2961E088E00E9407
:100F70001E2961E087E00E941E2960E082E00E9455
:100F80001E2961E084E00E941E29089542E050E09D
:100F900068E476E080E00E94A1270895E3E0F0E0B5
:100FA00089E080935700E491E67081E0E63009F033
:100FB00080E00895CF93DF93C82F0E94CE07882347
:100FC00081F0DFB781E080937005F8940E945706A6
:100FD00088E180936000C0936000C1110E945706B1
:100FE000DFBFDF91CF9108958F929F92AF92BF9212
:100FF000CF92DF92EF92FF92CF93FC01C0A5EC2F2E
:10100000E770F0E0E658FC4FA081B0E0C7FF03C0F6
:1010100024E130E002C02FE030E0FC0197A183E141
:10102000989FF0011124E25CFE4F80809180A280A5
:10103000B380A20FB31F20E43FE14DE750E00E94D0
:101040009D2DA50194010E94C92D8C2F887149F412
:1010500069017A01E0EDCE0EE7E0DE1EE11CF11C35
:101060001BC0C7FF05C060E47AE88CE29EE004C0C4
:1010700060E07EEE8AEB9BE069017A01F8EBCF0E2F
:10108000FBE0DF1EE11CF11CA50194010E94C92DAB
:10109000C20ED31EE41EF51EC701B60169517C4F76
:1010A0008F4F9F4F28EE33E040E050E00E94C92D63
:1010B000A8EEB3E00E94922DCF91FF90EF90DF90C9
:1010C000CF90BF90AF909F908F9008958F3F9105E4
:1010D00051F048F0811522E0920738F081159340D5
:1010E00030F482E0089580E0089581E0089583E07F
:1010F0000895A0E0B0E0EFE7F8E00C94152EEB01C6
:101100008A01B82FB695A0E028813981F8012083A3
:101110002A813B8121832C813D8122832E813F8145
:101120002383688179814A815B812C813D81EE81B5
:10113000FF819F2F9295990F990F907C272F2370F5
:10114000922B252F2370220F220F922B232F2370F7
:101150002295207F922BF80194830B5F1F4F2896D6
:10116000AF5FBA1788F680FF24C0888199810E94FA
:101170006608D82E8A819B810E946608E82E8C81A1
:101180009D810E946608F82E8E819F810E946608CC
:10119000F0E4DF9EA001112490E1E99E900111246A
:1011A000242B282BE4E0FE9EB0011124262BF8010D
:1011B0002083CDB7DEB7E7E00C94312E803223E0F8
:1011C000920708F1883E23E0920740F48F51934044
:1011D000E4E096958795EA95E1F70895803D27E04C
:1011E000920718F48C5D93400895883928E092079F
:1011F00068F4885C974074E0969587957A95E1F756
:101200008D509C4F089580E090E008958FEF93E01B
:1012100008958C30910540F4A4E0880F991FAA9599
:10122000E1F7885D9C4F0895843F23E0920718F40E
:1012300084529C4F0895811524E0920740F486570C
:10124000934FF4E0880F991FFA95E1F7089580E92C
:1012500098E008959C013695279525753575821B74
:10126000930B9C0123733373969587959695879579
:1012700083739373820F931F9C0154E036952795D7
:101280005A95E1F7280F391F2F703F7041E051E068
:10129000249FC001259F900D349F900D1124892F0C
:1012A00008955F98882319F00000289A02C0000072
:1012B000289800005F9A000008955F9A000083B1AB
:1012C0005F980000869581700895CF93DF93D82FA3
:1012D0005C9A5F985C98C8E08D2F80780E945109D5
:1012E000DD0FC150C9F75F98DF91CF9108958F77D7
:1012F0000E9465090895CF93DF93D82FC8E08D2F02
:1013000080780E945109DD0FC150C9F75F98DF91C5
:10131000CF910895CF93DF935F98C8E080E0D82FF6
:10132000DD0F0E945D098D0FC150C9F7DF91CF918C
:1013300008950E9477090E948A095C9A0895A1E0A5
:10134000B0E0E5EAF9E00C941A2E806869830E9407
:1013500065096981862F0E947B095C9A2196E2E0EB
:101360000C94362ECF93C0917D05C827E82FF0E06E
:10137000EC58FA4F678589E70E949F096C2F8DE32F
:101380000E949F096C2F82E40E949F09CF910895CB
:1013900086E20E9499090895CF93DF93EC016C8156
:1013A0008CE10E949F096D818DE10E949F096E81F1
:1013B0008EE10E949F096F8180E20E949F096885EB
:1013C00081E20E949F09698582E20E949F096A85E5
:1013D00083E20E949F096B8584E20E949F096C85CD
:1013E00085E20E949F096D858AE20E949F096E85B1
:1013F0008EE60E949F096F858FE60E949F0968898B
:1014000080E70E949F09698981E70E949F096A8994
:1014100082E70E949F09DF91CF910895CF92DF92DA
:10142000EF92FF92CF93DF936B017C01C11488E3AD
:10143000D8068CE9E8068CE1F80628F5C701B60164
:1014400020E836E948E950E00E94C92DE901689793
:1014500060E879E687E69FEF0E94A52D6C0D7D1D63
:101460008E1D9F1DF2E0660F771F881F991FFA954A
:10147000D1F721E732E040E050E00E94C92DF22E82
:10148000E32E80E421C0C701B60120E03DE241E344
:1014900051E00E94C92DE901689760E073ED8EEC80
:1014A0009EEF0E94A52D6C0D7D1D8E1D9F1D660F4C
:1014B000771F881F991F21E732E040E050E00E942B
:1014C000C92DF22EE32E80E66C2F6F71680F85E731
:1014D0000E949F096E2D86E70E949F096F2D87E766
:1014E0000E949F09DF91CF91FF90EF90DF90CF9006
:1014F0000895682F8DE60E949F0908958F929F920C
:10150000AF92BF92CF92DF92EF92FF92CF93DF9391
:10151000D82F83E00E94990980936F0584E00E9490
:10152000990980936E0560E086E00E949F0961E062
:1015300087E00E949F096FE789E00E949F0965E0AC
:101540008AE00E949F0962E18BE00E949F0965E1A9
:101550008CE00E949F096DEF8DE00E949F0960E082
:101560008EE00E949F09DD2319F08BE291E008C014
:1015700020919B0533E1239FC0011124825C9E4F83
:101580000E94CC096CE880E30E949F096FE082E32F
:101590000E949F0962E483E30E949F0980919C0559
:1015A00087FF02C064E101C06AE084E30E949F09F2
:1015B0006AE285E30E949F096DE286E30E949F092B
:1015C00064ED87E30E949F0960E088E30E949F0921
:1015D00060E089E30E949F09D11109C0C0907D0598
:1015E000D0907E05E0907F05F090800507C0C5E9AA
:1015F000CC2EC1ECDC2EED2CCEEDFC2ECAE38F2CD4
:101600009924AA24BB24682D8C2F0E949F09682D41
:1016100085E08C0F0E949F09FE2CED2CDC2CCC2445
:10162000CF5FCE3361F76FEF83E40E949F096FEFC6
:1016300084E40E949F096FEF85E40E949F096FEF89
:1016400086E40E949F09DD2311F066E002C06091EC
:1016500081058DE60E949F0960E089E70E949F094D
:10166000609182058AE70E949F0960E083E70E94FB
:101670009F0960E084E70E949F09D11109C0609131
:10168000790570917A0580917B0590917C0504C065
:1016900060E071EA8CEB93E30E940E0ADF91CF9138
:1016A000FF90EF90DF90CF90BF90AF909F908F9082
:1016B000089561E087E00E949F0964E28EE70E943E
:1016C0009F0963E088E00E949F0960E088E00E9433
:1016D0009F0965E087E00E949F0962E085E00E9423
:1016E0009F0983E00E94990980936F0584E00E941E
:1016F000990980936E05089583E00E94990980936B
:101700006F0584E00E94990980936E0561E087E08F
:101710000E949F096AE070E080E090E00E949428B7
:101720000E94590B00000895CF92DF92FF920F9311
:101730001F93CF93DF931F92CDB7DEB7082F162FDD
:101740008EE399830E949F09F02EC02E9981D92E95
:101750008C2D8F19811738F4F60161916F018FE795
:101760000E949F09F5CF64E085E00E949F0983E015
:101770000E94990980936F0584E00E9499098093E3
:101780006E050E94712860936A0570936B058093C3
:101790006C0590936D0569E087E00E949F0981E0E8
:1017A000809371050F90DF91CF911F910F91FF9062
:1017B000DF90CF9008950F931F930E94940B809118
:1017C0007105813099F40E94712800916A05109189
:1017D0006B0520916C0530916D05601B710B820BC0
:1017E000930B603A76488140910548F380917105EA
:1017F000813031F46EE971E080EE95E00E945D2A5F
:101800001F910F9108950F931F938091710582305E
:1018100021F41092710581E020C080917105813022
:10182000D9F40E94712800916A0510916B052091EE
:101830006C0530916D05601B710B820B930B613A47
:1018400076488140910540F061E087E00E949F0961
:101850001092710582E001C080E01F910F91089500
:10186000CF93DF93EC014AE050E06D2F70E080EE03
:1018700095E00E942B2B6EE280EE95E00E942F2ACD
:10188000BE0184E0769567958A95E1F76F707727BA
:101890004AE050E080EE95E00E942B2B6EE280EE55
:1018A00095E00E942F2ABE016F7077274AE050E032
:1018B00080EE95E00E942B2BDF91CF910895D82FD9
:1018C000C0E0CD1780F42D9A64E670E080E090E0EF
:1018D0000E9494282D9864E670E080E090E00E94D9
:1018E0009428CF5FEECF6CE271E080E090E00E9440
:1018F0009428E6CF0F931F93CF93DF93EC01062F2D
:1019000015E0115051F0CE010E942630081741F029
:10191000602FCE010E942E30F4CF82E00E945F0C37
:10192000DF91CF911F910F910895A0E0B0E0EBE916
:10193000FCE00C940C2E482E562EC0E0D0E0612C1A
:10194000712CE12CF12C00E010E041100CC06090F3
:10195000D20586E4689E3001112459E1E52EF12C70
:1019600008EB15E01EC091E049120FC06090D2054F
:10197000E6E46E9E30011124FBE16F0E711C49E21A
:10198000E42EF12C04E715E00CC082E0481209C0F7
:1019900028E1622E77247394EE24E394F12C01ED78
:1019A00015E043018C0E9D1E109273051092720576
:1019B0003401A62CA818B12CC30101966C01AE14F9
:1019C000BF04A8F4A00EB11E511006C0C3010E94AE
:1019D0002630F501808305C0F5016081C3010E94B6
:1019E0007A0CF50180810E9461063601E2CFC301C5
:1019F000511018C0C3010E942630B82EC6010E94A3
:101A000026302B2D30E0322F2227282B8091720593
:101A1000909173058217930779F4C0E0D0E05524C4
:101A2000539493CF3601609173050E947A0C6091B4
:101A30007205C6010E947A0CC05EDE4FC13E92E084
:101A4000D90708F482CF852DCDB7DEB7E0E10C943D
:101A5000282E61E082E00E94950C089560E082E00B
:101A60000E94950C8091D105853020F01092D1050F
:101A70000E94290D8091D1058093D205089561E0DF
:101A800080E00E94950C61E081E00E94950C089531
:101A900060E080E00E94950C882351F060E081E0D6
:101AA0000E94950C882321F080917405883349F0B9
:101AB0000E94BF060E947A0681E00E94DF060E9413
:101AC0003F0D0895882319F06AEA71E002C06EEABA
:101AD00071E080EE95E00E945D2A0895FF920F93D9
:101AE0001F93CF93DF9369EC7BE080EE95E00E943B
:101AF000092A4091790550917A0560917B05709192
:101B00007C052AE030E080EE95E00E94322B63EB0A
:101B10007BE080EE95E00E94092A40917D0550917E
:101B20007E0560917F057091800520E130E080EEB8
:101B300095E00E94322B6DE97BE080EE95E00E94FB
:101B4000092A4AE050E06091810580EE95E00E940C
:101B50005A2B67E87BE080EE95E00E94092A4AE074
:101B600050E06091820580EE95E00E945A2B61E77B
:101B70007BE080EE95E00E94092AC3E8D5E0F12CD5
:101B80008E0188818823A9F0FF2031F061EB71E09C
:101B900080EE95E00E942C2A21964AE050E0F80160
:101BA000608180EE95E00E94232BF394F8E1FF1210
:101BB000E7CF80EE95E00E94372A6BE57BE080EE70
:101BC00095E00E94092A4AE050E060919B0580EE72
:101BD00095E00E945A2B66E47BE080EE95E00E943F
:101BE000092AE0919C05E770F0E0EE0FFF1FEE5729
:101BF000FC4F6081718180EE95E00E945D2A61E377
:101C00007BE080EE95E00E94092A80919C05887116
:101C1000883069F028F4811113C068E27BE00CC0C1
:101C2000803141F0883161F46CE07BE005C06CE10B
:101C30007BE002C066E17BE080EE95E00E944B2AEB
:101C400068EF7AE080EE95E00E94092A40917505E0
:101C50005091760560917705709178052AE030E023
:101C600080EE95E00E94322B6FED7AE080EE95E0F9
:101C70000E94092A8091BD0580710E94620D66EC68
:101C80007AE080EE95E00E94092A8091BD0580747B
:101C90000E94620D6DEA7AE080EE95E00E94092ACA
:101CA0008091BD0580720E94620D60E97AE080EE4D
:101CB00095E00E94092A84E795E00E94F407AB01B1
:101CC000BC012AE030E080EE95E00E94142B6BE826
:101CD0007AE080EE95E00E94092A84E795E00E9470
:101CE000F4079B01AC0160E472E48FE090E00E9495
:101CF000C92DBA01A9012AE030E080EE95E00E94EA
:101D0000142B68E87AE080EE95E00E944B2ACDB76C
:101D1000DEB7E5E00C94332E8F929F92AF92BF9284
:101D2000CF92DF92EF92FF92811107C06FE77AE0C6
:101D300080EE95E00E944B2A2FC090E00E9474072D
:101D400024E630E040E050E00E94C92DCA01B9010C
:101D50002AE030E040E050E00E94C92D49015A01DC
:101D60006B017C012AE030E0B501A40180EE95E032
:101D70000E94142B6EE280EE95E00E942F2A2AE04A
:101D800030E0B701A60180EE95E00E94142B63E7D6
:101D900080EE95E00E946F2AFF90EF90DF90CF9049
:101DA000BF90AF909F908F9008951F93CF93DF9334
:101DB00065E77AE080EE95E00E94092A80919D0512
:101DC000813041F46CE57AE080EE95E00E944B2A88
:101DD00010E050C0823019F465E47AE0F5CF843029
:101DE00019F461E37AE0F0CF853091F766E27AE0AA
:101DF000EBCFC12FD0E0C930D1050CF441C068E36E
:101E0000610F80EE95E00E942F2A6EE17AE080EE6D
:101E100095E00E94092ABE016F5F7F4F4AE050E0C3
:101E200080EE95E00E94F32A63E17AE080EE95E08F
:101E30000E94092AC356DA4FE981E03218F566E0BC
:101E40007AE080EE95E00E94092A8981803130F0A5
:101E50006DE673E080EE95E00E942C2A69816F7038
:101E600070E06F5F7F4F4AE050E080EE95E00E94A7
:101E7000FC2A1F5F80914605181708F4BACF0FC0DF
:101E800061E3BECFEF70F0E0EE0FFF1FEE56FC4FA8
:101E90006081718180EE95E00E945D2AEACF6BEE51
:101EA00079E080EE95E00E94092A8091B5050E94B4
:101EB0008C0E60ED79E080EE95E00E94092A809119
:101EC000B6050E948C0E65EB79E080EE95E00E94ED
:101ED000092A8091B7050E948C0E6AE979E080EEAC
:101EE00095E00E94092A4091AD055091AE056091A0
:101EF000AF057091B005411551056105710539F1C6
:101F00002AE030E080EE95E00E94322B67E679E02F
:101F100080EE95E00E94092A8091B1050E94990700
:101F2000AB01BC012AE030E080EE95E00E94322B4C
:101F300063E479E080EE95E00E94092A4AE050E0EF
:101F40006091B20580EE95E00E945A2B06C06AE3CC
:101F500079E080EE95E00E944B2A6DE179E080EE19
:101F600095E00E94092A6091B3057091B4054AE09A
:101F700050E080EE95E00E94442B60E079E080EE36
:101F800095E00E94092A6091AC05603450F470E03D
:101F90006F5F7F4F4AE050E080EE95E00E94FC2AA0
:101FA00006C067EF78E080EE95E00E944B2A6AED6C
:101FB00078E080EE95E00E94092A8091AB0580FFD1
:101FC00003C063EB71E002C067EB71E080EE95E067
:101FD0000E945D2A6DEB78E080EE95E00E94092A70
:101FE0008091AB0582700E94620D6EE978E080EE10
:101FF00095E00E94092A8091AB0584700E94620DD1
:102000006FE778E080EE95E00E94092A8091AB05A9
:1020100088700E94620DDF91CF911F9108950F93F8
:102020001F93CF93DF93209143052F3FA9F56FEFC7
:1020300075E080EE95E00E94092A82E893E00E9414
:10204000300C6EED75E080EE95E00E94092A8091DB
:102050004405909145050E94300C6BEA75E080EED6
:1020600095E00E944B2A68E875E080EE95E00E94BA
:102070004B2A60E775E080EE95E00E944B2A6BE406
:1020800075E080EE95E00E944B2A80EE95E00E947C
:10209000372A0E94D50E68C012160CF065C033278F
:1020A00027FD30958091460590E0821793070CF448
:1020B0005BC066E375E080EE95E00E94092A6091BE
:1020C0004305772767FD70954AE050E080EE95E084
:1020D0000E94FC2A6BE075E080EE95E00E94092AE0
:1020E00010E008E2809147051817D0F5C12FD0E025
:1020F000CC0FDD1FC85BDA4F288130E080914305AB
:10210000992787FD909501972817390739F56BEBCB
:1021100071E080EE95E00E942C2A4AE050E0602FAA
:1021200080EE95E00E94232B6FEB71E080EE95E04E
:102130000E942C2AE981EF70F0E0EE0FFF1FEE56AF
:10214000FC4F6081718180EE95E00E942C2A63EC47
:1021500071E080EE95E00E942C2A0F5F1F5FC2CFD6
:1021600080EE95E00E94372ADF91CF911F910F9169
:102170000895FF920F931F93CF93DF93C3E8D5E0A9
:10218000F12C8E0188818823D1F165EC71E080EE1D
:1021900095E00E942C2A4AE050E06F2D80EE95E0F9
:1021A0000E94232B62ED71E080EE95E00E942C2AC4
:1021B0002196F801208130E0A0E1B7E20E94832D52
:1021C0009B01AC01A0918205B0E00E94922DAB0171
:1021D000BC018091790590917A05A0917B05B09121
:1021E0007C05480F591F6A1F7B1F2AE030E080EEF4
:1021F00095E00E94322BF394F8E1FF12C2CFCDB7E5
:10220000DEB7E5E00C94332E1092DD0485E6EEEDAA
:10221000F4E0DF011D928A95E9F70895CF93C82F66
:102220008F3719F0883009F045C0E091DD04EE23C6
:10223000D9F1E150E093DD04F0E0E252FB4F10826F
:102240006DE070E080EE95E00E945906C0E080915C
:10225000DD04C81760F4EC2FF0E0E252FB4F608120
:1022600070E080EE95E00E945906CF5FF0CF60E20B
:1022700070E080EE95E00E9459066DE070E080EE1F
:1022800095E00E945906C0E08091DD04C81778F5FA
:10229000EC2FF0E0E252FB4F608170E080EE95E0C1
:1022A0000E945906CF5FF0CF67E080EE95E00E9474
:1022B0002F2A1DC08B3119F40E9404111AC08D30D1
:1022C000C1F08A30B1F08091DD04843668F76C2F5C
:1022D00070E080EE95E00E945906E091DD0481E017
:1022E0008E0F8093DD04F0E0E252FB4FC08380E06C
:1022F00001C081E0CF910895CF93C82F0E9471282B
:102300006093C6047093C7048093C8049093C90473
:10231000C093DB04CC2329F040E051EE60E070E094
:1023200004C040E855E260E070E080EE95E00E9475
:10233000B92CCF9108959091CA04492F4F7050E065
:10234000BA016F5F7F4F292F30E0E4E03595279584
:10235000EA95E1F76217730759F0FA01E553FB4F6D
:10236000808381E0890F8F70907F892B8093CA04CE
:1023700008956EE770E080EE95E00E94590608959A
:10238000A3E1B1E0E6ECF1E10C940D2EE3E8F5E019
:10239000712C8191882321F0739428E17212F9CF76
:1023A00066ED71E080EE95E00E945D2A4AE050E023
:1023B000672D80EE95E00E945A2B80E00E947E0AF5
:1023C0000E94590B8E010E5F1F4FC12CD12C76013C
:1023D000C39466246A945C2C0E9465284B015C01BE
:1023E0002091820530E0A0E1B7E20E94832D9B019D
:1023F000AC01C701B6010E94A52D2091790530914D
:102400007A0540917B0550917C05620F731F841FF4
:10241000951F2091B9053091BA054091BB055091A7
:10242000BC05261737074807590718F4F8016082DA
:1024300025C08C2D0E94B20961E070E080E090E040
:102440000E949428F80110820E9465286819790971
:102450008A099B09643F71408105910540F40E94FF
:10246000C809F8019081981778F78083EDCF50FE66
:1024700003C02C982D9A02C02C9A2D982FEFC21AC7
:10248000D20AE20AF20A0F5F1F4F8FEFC816D1047B
:10249000E104F10409F09FCFCE019395FC01D82E01
:1024A0007FEF68EC2E2F281B271510F051E056C047
:1024B000DE01129651E02FEF41E03D91321710F00E
:1024C000322F01C0452F5F5F5F3F11F0232FF5CF03
:1024D0004193242F30E0A1E0B0E0AC0FBD1FA20F6C
:1024E000B31F5C93413079F0DE01A20FB31F5C9300
:1024F000423049F0AFEFBFEFAC0FBD1FA20FB31FCB
:102500006C934E3F78F6A2E0B0E0AC0FBD1FA20F77
:10251000B31F7C934D3F30F6A3E0B0E0AC0FBD1F7E
:10252000A20FB31F6C93BECF452F242F30E0FC01C8
:10253000E20FF31F6081AFEFB0E0AC0FBD1FA20F41
:10254000B31F2C91621748F44150DC01A40FB11D58
:102550002C9120836C934111E8CF5F5F571520F3D6
:10256000372D369520E0231770F4DC01A20FB11D42
:102570004C91522F530FFC01E50FF11D50815C93DC
:1025800040832E5FF0CFF3E8EF2EF5E0FF2E8C01B5
:10259000802F8D19871598F4F801C1908F014AE0BA
:1025A00050E06C2D80EE95E00E94232B6CE280EED3
:1025B00095E00E942F2AF701C1927F01E9CF80EEBA
:1025C00095E00E94372A81E0CD5EDE4FEFE00C946B
:1025D000292E1F920F920FB60F9211240F931F9363
:1025E0002F933F934F935F936F937F938F939F931B
:1025F000AF93BF93EF93FF934091BD055091BE05FC
:102600006091BF057091C00589B18A019B0100747A
:1026100011272227332783FB882780F990E0A0E049
:10262000B0E0081719072A073B0709F468C0809132
:102630008400909185001092850010928400209172
:10264000A70421115CC045FD02C096958795853C85
:1026500029E09207C0F180910A0190E0A0E0B0E08B
:102660000CE176956795579547950A95D1F74115F1
:1026700051056105710521F441E050E060E070E032
:10268000481759076A077B07D8F480910A018F3FE2
:10269000B9F040E080910A01481780F4842F90E05F
:1026A000880F991FFC01E957FB4F20813181FC0104
:1026B000E55FFE4F318320834F5FECCF1092A8047B
:1026C00010920A011CC08D3B22E09207A8F02091D5
:1026D0000A01203188F410910A0121E0210F209392
:1026E0000A010E94DE08E12FF0E0EE0FFF1FE9571C
:1026F000FB4F9183808303C08FEF80930A01FF918A
:10270000EF91BF91AF919F918F917F916F915F9169
:102710004F913F912F911F910F910F900FBE0F90EE
:102720001F90189583E0809380008AE18093810058
:102730008FEF9FEF909389008093880010926F0035
:1027400088E080936D00E8E6F0E08081846080831B
:1027500008950E942E0D8091D205843011F41092BC
:10276000D20508956F3018F086958058089589E055
:10277000689F802D11240895A0E0B0E0E2ECF3E121
:102780000C94142EC82F0E947128009138041091C7
:10279000390420913A0430913B046B017C01C01A4A
:1027A000D10AE20AF30A9701860149E8C41643E117
:1027B000D406E104F10410F010923C046093380454
:1027C0007093390480933A0490933B042091A704BA
:1027D0008FEF820F8230D8F5E0913C04EE2309F4AC
:1027E0004EC1E13011F482E0B8C1E03108F034C1EB
:1027F00081E08E0F80933C04F0E0E957FB4FC083EB
:10280000803109F0ACC1E9E8F4E0213029F4A1817C
:10281000A695A695808108C080819181A92FA69553
:10282000A695A69596958795A03148F4B0E090E0DE
:10283000AA0FBB1FA55FBE4F11969C938E9310925B
:10284000A804329684E0E739F807F9F688C1233006
:1028500009F005C1E0913C04E11104C0CF3009F05A
:102860007EC10DC1E83148F481E08E0F80933C04B5
:10287000F0E0EA57FB4FC08372C1E83109F0ECC0C9
:10288000C111EAC040E050E0ABE0CA01B3E0880FFC
:10289000991FBA95E1F7A49F9001A59F300D1124CF
:1028A000F901E957FB4F6081E1817E2F77707595C3
:1028B0006795FC01EE0FFF1FE55FFE4F718360839C
:1028C000F901E857FB4FB081B695B695B695E18111
:1028D000FE2FF295FF0FF07E6F2F6B2BE695E6959E
:1028E000E6957E2F777075956795FC01EE0FFF1FBB
:1028F000E35FFE4F71836083F901E757FB4FB081BF
:10290000B295B695B695B370C181DC2FDD0FDD0FA2
:102910006D2F6B2BC295C695C695C370E281E17091
:10292000EE0FEE0F7E2F7C2B75956795FC01EE0F59
:10293000FF1FE15FFE4F71836083F901E557FB4F95
:10294000B081B695E181FE2FF795FF27F7956F2FA0
:102950006B2BE6957E2F777075956795FC01EE0FD2
:10296000FF1FEF5EFE4F71836083F901E457FB4F59
:10297000B081B295BF70E181FE2FF295F07F6F2F8D
:102980006B2BE295EF707E2F777075956795FC0144
:10299000EE0FFF1FED5EFE4F71836083F901E35779
:1029A000FB4FB081BB1FBB27BB1FC181DC2FDD0FDD
:1029B0006D2F6B2BCC1FCC27CC1FE281E370EE0F69
:1029C0007E2F7C2B75956795FC01EE0FFF1FEB5E4C
:1029D000FE4F71836083F901E157FB4FB081B695DB
:1029E000B695E181FE2FF295FF0FFF0FF07C6F2F60
:1029F0006B2BE695E6957E2F777075956795FC01B4
:102A0000EE0FFF1FE95EFE4F71836083F901E0570F
:102A1000FB4F20812295269527703181E32FEE0F01
:102A2000EE0FEE0F6E2F622B732F729576957770E7
:102A300075956795FC01EE0FFF1FE75EFE4F7183F2
:102A400060834F5F5F4F4230510509F01ECF809188
:102A50009D0483FF1092A80410923C0480C024308F
:102A600009F07DC060913C0461110BC0C83AB1F41B
:102A7000109273051092720588EA0E94610681E047
:102A80006CC0613019F4C093370404C0623031F473
:102A9000C09336048C2F0E9461065AC0E091360420
:102AA0002E2F30E0220F331F462F50E0C90102962F
:102AB000841795073CF0633268F7FA01EC57FB4F37
:102AC000C083E8CF2D5F3F4F8C2F90E0609172055F
:102AD000709173054217530749F4982F882786276A
:102AE0009727909373058093720532C06817790712
:102AF00069F580913704813049F5E13118F080E1C2
:102B000080933604F0903604C8E8D4E000E010E08A
:102B10000F15D0F4FE013197808190E0982F88271F
:102B20002881822B43E0969587954A95E1F70E948C
:102B3000DE08F801EE0FFF1FE55FFE4F91838083F3
:102B40000F5F1F4F2296E4CF1092A80410923C040E
:102B500080913C04882319F08F5F80933C04CDB7AB
:102B6000DEB7E8E00C94302EE82FF0E0E854FA4F9E
:102B7000E185E03150F4F894F0E0EE0FFF1FE55FDF
:102B8000FE4F8081918178940895E03121F0E13108
:102B900031F483E101C082E10E94B329089580E00D
:102BA00092E00895A2E2B0E0E8EDF5E10C940A2E7F
:102BB0009E012F5F3F4F80E1D9011D928A95E9F771
:102BC00064E072E080EE95E029A33AA30E945D2ABA
:102BD0000E947C0B1D8A1E8A1F8A188E312C212C84
:102BE00000E0812C912C5401412C74E7572E7BE896
:102BF000672E72E3772EE0E5CE2EE3ECDE2EE12C9D
:102C0000F12C84EF91E0A0E0B0E08D8F9E8FAF8F2C
:102C1000B8A380E09EECADEEB4E3898F9A8FAB8FC2
:102C2000BC8F80E094E7ABE8B2E3898B9A8BAB8BE7
:102C3000BC8B80EE95E00E94712B892B09F4E1C0DA
:102C400080EE95E00E949E2B9C0133272C323105AB
:102C500009F442C0ACF42332310509F0ABC019824B
:102C60001A821B821C821D821E821F821886198670
:102C70001A861B861C861D861E861F86188A60C0C3
:102C80002434310529F02335310509F4B2C092C04E
:102C900064E480EE95E00E942F2A2AE030E040E0D4
:102CA00054E76BE872E380EE95E00E94BD2A6CE287
:102CB00080EE95E00E942F2A2AE030E040E05EECB2
:102CC0006DEE74E380EE95E00E94BD2A6CE280EE2A
:102CD00095E00E946F2AADCF0F5F043009F0A9CFB5
:102CE00029813A814B815C81A8EEB3E00E94922D4C
:102CF000698B7A8B8B8B9C8B2D813E814F81588584
:102D00000E94922D698F7A8F8B8F9C8F29853A85AF
:102D10004B855C852D8F3E8F4F8F58A32D853E852B
:102D20004F8558890E94922D6B017C0160323EE4F0
:102D300073078105910530F462E38CE10E949F09DD
:102D400000E077CF603345E774078105910510F403
:102D500062E2F3CF60345CE975078105910510F4F8
:102D600066E2EBCF80E5C81683ECD806E104F104F7
:102D700010F462E1E2CF90E6C9169AEED906E104BA
:102D8000F10410F465E1D9CFA0E7CA16A1E1DA0693
:102D9000A1E0EA06F10410F461E0CFCFB0EACB166F
:102DA000B6E8DB06B1E0EB06F10410F463E0C5CF52
:102DB00065E0C3CF10ED180F1A3008F03ACFE1E00C
:102DC000F0E0EC0FFD1F24E0029FE00DF11D112447
:102DD0002081318142815381AAE0B0E00E94922D8E
:102DE000610F711D811D911D6083718382839383A7
:102DF00020CF49885A886B887C88812C912C54017B
:102E000018CF81149104A104B10489F4C301B20163
:102E10000E940E0A61E070E080E090E00E94942839
:102E20001D8A1E8A1F8A188E312C22242A948D8D89
:102E30009E8DAF8DB8A188169906AA06BB06D0F460
:102E40000E94C8092D893E894F89588D280F311D50
:102E5000411D511D2D8B3E8B4F8B588F381608F41A
:102E6000382E821508F4282E3FEF831A930AA30AFE
:102E7000B30A56C0C301B20128EE33E040E050E08F
:102E80000E94C92DBA01A9012AE030E080EE95E048
:102E90000E94142B6CE280EE95E00E942F2A4AE0FB
:102EA00050E0632D80EE95E00E94232B6CE280EED3
:102EB00095E00E942F2A6D897E898F89988DA501C2
:102EC00094010E94C92DBA01A9012AE030E080EEE8
:102ED00095E00E94142B6CE280EE95E00E942F2A70
:102EE0004AE050E0622D80EE95E00E94232B6CE2D8
:102EF00080EE95E00E946F2A4C0C5D1C6E1C7F1CBE
:102F0000898D9A8DAB8DBC8D84159505A605B70569
:102F100020F449885A886B887C88812C912C540134
:102F200029893A894B895C89283E334041055105FE
:102F300009F07FCEA296E2E10C94262EACE1B0E03F
:102F4000E4EAF7E10C94142E0E9471286B017C01D5
:102F500081E00E947E0A14E703E0198361E0CE015C
:102F600001960E94DB0B009371050E94590B6AEFDA
:102F700070E080E090E00E94942880917105833099
:102F800089F480EE95E00E94712B892B59F40E9400
:102F900071286C197D098E099F096038734C894C22
:102FA0009140D8F280917105833009F44FC08FE7CA
:102FB0000E9477090E948A098983843511F083E091
:102FC0005CC00E948A0910924405809345050E94C6
:102FD0008A092091440530914505280F311D309311
:102FE0004505209344050E948A09809346050E9466
:102FF0008A0980934705813110F7F12C0F2D10E0DD
:103000008091470590E0880F991F0817190740F431
:103010000E948A09F801E85BFA4F8083F394EECFAF
:1030200080E7898361E0CE0101960E94DB0B83E09B
:10303000809371050E94590B62E370E080E090E09C
:103040000E94942880917105833011F482E015C0AC
:103050008FE70E9477090E948A098983803509F0E9
:10306000AECF0DE915E00E948A09F80181938F0126
:10307000F5E0083B1F07B9F781E06C96E8E00C9497
:10308000302E80914305992787FD9095A92FB92F60
:10309000FC013196EB30F10508F066C0EC5CFF4FA7
:1030A0000C94412E62E778E080EE95E00E944B2A76
:1030B00082E893E00E94300C6AE578E080EE95E0CB
:1030C0000E944B2A65E378E080EE95E00E944B2A4F
:1030D0006BE078E080EE95E00E944B2A6AEE77E0A4
:1030E00080EE95E00E944B2A6DEB77E080EE95E054
:1030F0000E944B2A67E977E080EE95E00E944B2A18
:1031000063E777E080EE95E00E944B2A6CE477E07D
:1031100080EE95E00E944B2A80EE95E00E94372ACF
:103120000E946E0D21C06FE277E01AC06AE077E07E
:1031300017C065EF76E014C066ED76E011C062E975
:1031400076E00EC06DE776E00BC068E676E080EED4
:1031500095E00E944B2A62E276E002C06CE076E0E5
:1031600080EE95E00E944B2A6AE070E080E090E0FB
:103170000E94942880EE95E00E94712B892B29F003
:1031800080EE95E00E949E2BF5CF0895ACE1B0E073
:10319000ECECF8E10C94142E909143059F3F09F05C
:1031A00023C1482F50E0FA013A97EF36F10508F0B5
:1031B0000FC1E15CFF4F0C94412E61E172E0A0C0B1
:1031C0006DE172E080EE95E00E945D2A85E78983DB
:1031D0008BE1EDE9F5E0DE01129601900D928A9502
:1031E000E1F76CE1CE0101960E94DB0B0E94590BC6
:1031F00083E08093710568EC70E080E090E00E94CD
:10320000942880917105843009F0E2C08FE70E9414
:1032100077090E948A098983853509F0D9C06DEE46
:1032200074E080EE95E00E944B2A6FEC74E080EE33
:1032300095E00E944B2A61EB74E096C065E372E072
:1032400080EE95E00E945D2A89E6898361E0CE01E7
:1032500001960E94DB0B0E94590B83E0809371055D
:1032600068EC70E080E090E00E9494288091710505
:10327000843009F0ADC08FE70E9477090E948A0967
:1032800089838E010E5F1F4F7E014DE1E40EF11C1C
:103290000E948A09F80181938F01EE15FF05C1F79D
:1032A0008BE1FE013296ADE9B5E001900D928A9571
:1032B000E1F78981893409F08BC063E974E080EE1D
:1032C00095E00E944B2A65E774E080EE95E00E944D
:1032D0004B2A67E574E048C06FE472E080EE95E049
:1032E0000E945D2A8EEF8093430572C08052875002
:1032F000805390914605981708F066C06EE572E01D
:1033000080EE95E00E945D2A63C084E180934305CE
:1033100060E274E029C085E18093430569EE73E0C3
:1033200023C086E18093430562EB73E01DC087E113
:103330008093430568E673E017C088E180934305F6
:1033400067E573E011C089E18093430563E473E0AE
:103350000BC08AE1809343056EE273E005C08BE108
:103360008093430566E073E080EE95E00E944B2A6F
:103370002FC06CEE72E080EE95E00E944B2A8091A7
:10338000AB0591E01DC066ED72E080EE95E00E9415
:103390004B2A8091AB0592E013C061EC72E080EEA5
:1033A00095E00E944B2A8091AB0594E009C066EA43
:1033B00072E080EE95E00E944B2A8091AB0598E088
:1033C00089278093AB058FEF809343050E940F10F0
:1033D00080EE95E00E94712B892B09F45AC180EE92
:1033E00095E00E949E2BF4CF0E940E11882309F4D1
:1033F00050C18091DD04811104C08FEF809343059B
:1034000040C140E050E060E070E08EED94E00E944A
:10341000B82E40914305042F112707FD1095212F49
:10342000312FF8013197EB31F10508F01AC1E2555F
:10343000FF4F0C94412E552747FD5095209146058E
:1034400030E0241735070CF40CC18B019C010150AE
:10345000110921093109003211052105310558F002
:10346000C0904705E9E4F5E0F12CD12CA8E2EA2E62
:10347000415051090FC0FA01E356FA4F6150608381
:10348000D8C0DF0111972C9130E02417350729F0BF
:10349000F3943296FC10F5CFCAC00E2D10E020E058
:1034A00030E0061717072807390741F42081DA01B1
:1034B000A356BA4F11962C93DD24D394E394E8CF0E
:1034C0006F3F71058105910511F008F0CAC0609346
:1034D000B505AFC06F3F71058105910511F008F08A
:1034E000C0C06093B605A5C06F3F71058105910509
:1034F00011F008F0B6C06093B7059BC02091DE04C0
:1035000020622037E9F440E050E060E070E08FEDA9
:1035100094E00E94B82E9B01AC01DC01CB01019725
:10352000A109B1090897A105B10508F0ADC0A4ED46
:10353000B0E30E94922D6A5E7C4A8A46954E24C072
:103540002636E9F440E050E060E070E08FED94E072
:103550000E94B82E9B01AC01DC01CB010197A109AF
:10356000B1090797A105B10508F08EC0A8EAB1E638
:103570000E94922D645E7C438E46944E05C0611578
:1035800071058105910571F08B019C0114572B4841
:1035900032430130FAE51F07F2E62F07F2E03F075A
:1035A00008F05FC06093AD057093AE058093AF05E2
:1035B0009093B0053EC06F3F71058105910511F0F4
:1035C00008F04FC06093B10534C08B019C010150DD
:1035D0001109210931090F3F11052105310508F0B5
:1035E00040C06093B20525C08B019C01045C19406A
:1035F000210931090D344DE114072105310528F465
:103600007093B4056093B30514C06115710581050D
:10361000910521F48FEF8093AC050BC061347105E7
:1036200081059105F0F461506093AC0502C0DD2086
:10363000C1F08091DC0481111AC080917D059091C8
:103640007E05A0917F05B09180050196A11DB11D59
:1036500080937D0590937E05A0937F05B0938005B0
:1036600006C060E772E080EE95E00E945D2A0E944D
:1036700004118FEF809343056AE080EE95E00E948D
:103680006F2A0E940F1005C061E070E080E090E0BA
:103690007BCF6C96E8E00C94302E6AE572E080EE09
:1036A00095E00E944B2A62E472E080EE95E00E9471
:1036B0004B2A80EE95E00E94712B892B31F080EE31
:1036C00095E00E949E2B0E94C6180E949E17823091
:1036D00029F0833051F46DE072E002C064E272E0E0
:1036E00080EE95E00E944B2A08958FEF809343056A
:1036F0001092DC040E940F10809143058E3F69F008
:1037000080EE95E00E94712B892BB1F380EE95E05D
:103710000E949E2B0E94C618EFCF08950F931F930F
:10372000109143051F3F09F0D2C0893409F457C0F6
:1037300000F5883309F469C058F4803309F477C080
:1037400008F061C08B3109F440C08132B1F1B9C0D9
:10375000813409F487C030F4893309F466C08034B9
:1037600061F1AFC0823409F48EC0863409F448C0D8
:10377000A8C0823609F487C078F4883531F128F47E
:103780008235C1F18335E1F09CC08A3509F494C0DB
:10379000813609F467C095C0823761F128F4863616
:1037A00079F18936E1F08DC0883779F08A3709F4EC
:1037B00083C0833709F085C003C061E172E015C0A2
:1037C0000E943F0D6EE872E004C00E94480D68EA56
:1037D00072E080EE95E00E945D2A8EEF70C00E943C
:1037E0007A060E94BF0667EC72E080EE95E00E94C8
:1037F0005D2A67C081E00E94DF0660EE72E0F5CFCF
:103800000E94B9105EC080535AC06AEF71E080EE2A
:1038100095E00E944B2A90919C0588E0890F887161
:10382000977E892B80939C051AC089E048C067EE7B
:1038300071E080EE95E00E944B2A8091BD05909149
:10384000BE05A091BF05B091C00520E182278093FD
:10385000BD059093BE05A093BF05B093C00510931E
:1038600043052FC061ED71E080EE95E00E944B2A88
:103870008091BD059091BE05A091BF05B091C00596
:1038800040E4842710C060EC71E080EE95E00E9477
:103890004B2A8091BD059091BE05A091BF05B091C6
:1038A000C00520E282278093BD059093BE05A093BA
:1038B000BF05B093C00502C00E944D1B8FEF8093DF
:1038C0004305809143058E3F09F0D4C0DDC00E94BE
:1038D0000E11882309F4D8C08091DD04811104C041
:1038E0008FEF80934305C6C040E050E060E070E099
:1038F0008EED94E00E94B82E00914305112707FD3C
:103900001095212F312FF8013197E930F10508F09A
:10391000B4C0E753FF4F0C94412E8B019C01015022
:1039200014472B4832430F3F19452246324008F0D6
:10393000A4C06093790570937A0580937B0590937A
:103940007C0577C060937D0570937E0580937F052D
:103950009093800581E08093DC046BC06830710532
:103960008105910508F089C06093810562C08B01D3
:103970009C0101501109210931090A301105210565
:10398000310508F07AC06093820553C061EB71E0A5
:103990008EED94E00E94F22F10E0009799F00E94C3
:1039A000CC2F009779F0183130F4E12FF0E0EC588B
:1039B000FA4F87871F5F61EB71E080E090E00E9423
:1039C000F22FEBCF1831A8F5E12FF0E0EC58FA4FC9
:1039D00017861F5FF7CF653071058105910508F0E7
:1039E0004CC060939B0525C08B019C0101501109BF
:1039F000210931090630110521053105F0F5209125
:103A00009C05287F262B20939C0513C08B019C01CD
:103A100001501109210931090115124C21403105CC
:103A200060F56093750570937605809377059093A4
:103A300078058091DC04811113C080917D059091FF
:103A40007E05A0917F05B09180050196A11DB11D55
:103A500080937D0590937E05A0937F05B0938005AC
:103A60000E9404118FEF809343056AE080EE95E099
:103A70000E946F2A0E94411807C060E772E080EE42
:103A800095E00E945D2AECCF1F910F9108958FEF72
:103A9000809343051092DC040E94411880914305F5
:103AA0008E3F69F080EE95E00E94712B892BB1F377
:103AB00080EE95E00E949E2B0E948E1BEFCF6AE065
:103AC00070E080E090E00E94942880EE95E00E94F3
:103AD000712B892B29F080EE95E00E949E2BF5CF6B
:103AE0000895CF93C82F682F80EE95E00E94CB2BCE
:103AF000909168059C2790936805CF910895A1E067
:103B0000B0E0E5E8FDE10C941A2E99830E94711D46
:103B10009981892F0E94711D2196E2E00C94362E26
:103B20001F93CF93DF93182FEB011092680565EB7D
:103B300070E080EE95E00E94590662E670E080EE4B
:103B400095E00E945906812F0E94711DCE010E94AE
:103B50007F1DDF91CF911F9108956091680580EEE0
:103B600095E00E94CB2B0895A1E2B0E0EAEBFDE1E5
:103B70000C94162E7B018A018C3009F453C108F095
:103B800040C0863009F4BCC018F5833009F491C0F8
:103B900070F4813009F472C0823009F048C26BE1E0
:103BA00070E082E00E94901D0DE915E078C084303D
:103BB00009F487C0853009F03AC26091470570E08A
:103BC000660F771F85E00E94901D08E415E086C00F
:103BD000893009F4A7C070F4873009F49BC088309D
:103BE00009F025C261E070E088E00E94901D80919C
:103BF000D20523C28A3009F4CAC08B3009F4F2C05E
:103C000016C28A3609F475C1D8F4873609F43AC168
:103C100038F4853609F40EC1863609F41FC107C28F
:103C2000883609F437C1893609F001C261E070E0D5
:103C300089E60E94901D0E947A060E94BF06F5C187
:103C40008D3609F4D4C138F48B3609F491C18C3621
:103C500009F49AC1ECC18E3609F4DCC1873C09F045
:103C6000E6C161E070E087EC0E94901D81E00E9457
:103C7000711D0E94AD1D10926905E3C169E270E0FB
:103C800081E00E94901D04E715E0F80181918F0109
:103C90000E94711DF5E00D391F07B9F7D0C1F80179
:103CA00081918F010E94711DF5E0083B1F07B9F754
:103CB000C6C161E070E083E00E94901D0E949E17E3
:103CC000BCC161E070E084E00E94901D81E00E9430
:103CD000711D0E94AD1D0E94D215B3C18091470590
:103CE00090E0880F991F980128543540281739070C
:103CF00008F0A5C1F80181918F010E94711DEECFDE
:103D000062E070E086E00E94901D82E893E00E94ED
:103D10007F1D95C161E070E087E00E94901D809159
:103D200046058BC186E6898361E0CE0101960E943B
:103D3000DB0B0E94590B83E08093710568EC70E007
:103D400080E090E00E949428809171058430D9F43D
:103D50008FE70E9477090E948A098983863469F473
:103D600060E270E089E00E94901D10E20E948A09E2
:103D70000E94711D1150D1F762C161E070E089E0CD
:103D80000E94901D52C161E070E089E053C169E179
:103D900070E08AE00E94901D81E08093B805209138
:103DA00070058091BD059091BE05A091BF05B091B1
:103DB000C005222311F0806801C08F778093BD0574
:103DC0009093BE05A093BF05B093C00508EB15E026
:103DD000F80181918F010E94711DF5E0013D1F07DF
:103DE000B9F72DC161E270E08BE00E94901D8091D7
:103DF000A8048F3F39F08091A80491E0980F909328
:103E0000A80402C08091A8040E94711D10E0812FB7
:103E10000E94B4150E9409090E947F1D1F5F103186
:103E2000B1F70DC161E070E08CE00E94901D8091BF
:103E3000D10503C161E070E085E60E94901D89E232
:103E4000E816F10409F0F8C0D801E4E7F5E08D9137
:103E5000819385E0ED39F807D1F7E7C061E070E0C4
:103E600086E60E94901DEBE1EE16F10409F0E4C035
:103E7000D801EDE9F5E08D91819385E0E83BF80705
:103E8000D1F7D3C061E070E087E60E94901D0E94E8
:103E90003F0DCBC061E070E088E60E94901D85E791
:103EA00089838BE1EDE9F5E0DE01129601900D9238
:103EB0008A95E1F76CE1CE0101960E94DB0B0E942E
:103EC000590B83E08093710560E273E080E090E03D
:103ED0000E94942880917105843009F0ADC08FE76D
:103EE0000E9477090E948A098983853509F0A4C058
:103EF0009CC061E070E08AE60E94901D89E689839B
:103F000061E0CE0101960E94DB0B0E94590B83E019
:103F10008093710560E273E080E090E00E94942855
:103F200080917105843009F087C08FE70E9477097E
:103F30000E948A0989838E010E5F1F4F7E01EDE189
:103F4000EE0EF11C0E948A09F80181938F01EE1593
:103F5000FF05C1F78BE1FE013296ADE9B5E00190B6
:103F60000D928A95E1F78981893409F065C05DC0B9
:103F700061E070E08BE60E94901DF80180818093E3
:103F8000D2050E94480D51C061E070E08CE60E94AD
:103F9000901DF0E2EF16F10461F487E6898380E278
:103FA000F801DE01129601900D928A95E1F761E227
:103FB00003C087E4898361E0CE0101960E94DB0B98
:103FC0000E94590B83E0809371056CE474E080E0FB
:103FD00090E00E94942880917105843069F58FE704
:103FE0000E9477090E948A09873431F51EC061E07A
:103FF00070E08DE60E94901D89E1E816F104E1F47D
:10400000D801E8EBF5E08D91819385E0E13DF8077B
:10401000D1F70BC061E070E08EE60E94901DF801C0
:1040200080818093D1050E94290D81E006C061E066
:1040300070E08AEC0E94901D80E00E94711D0E9439
:10404000AD1DA196E6E00C94322EA0E0B0E0EBE2CC
:10405000F0E20C94142ECAECD3E014E606E035E04E
:10406000F32E44E0E42E53E0D52E62E0C62E80EE1F
:1040700095E00E94712B892B09F49BC080EE95E09E
:104080000E949E2B282F809335044091340450E0E9
:104090004730510560F7FA01EE52FF4F0C94412E64
:1040A000853B29F781E080933404E1CF823609F023
:1040B0007DC0C0923404DBCF8093330480933204FC
:1040C000D0923404D4CF9C01332730933104209311
:1040D000300490913204982790933204E092340493
:1040E000C6CF382F22274091300450913104242B21
:1040F000352B30933104209330049091320498276B
:1041000090933204F09234042536310508F4AFCF91
:1041100061E070E08CEC0E94901D81E00E94711DB6
:104120000E94AD1D43C020912E0430912F04F9014F
:10413000E653FC4F80839091320498279093320489
:10414000C901019690932F0480932E04209130048E
:10415000309131048217930708F489CF0093340417
:1041600086CF8091320482130BC060912E0470912F
:104170002F044AEC53E0809133040E94B41D0DC01B
:1041800062E070E08BEC0E94901D809133040E94ED
:10419000711D809168050E94711DFE01812F119291
:1041A0008A95E9F710922F0410922E04109234048D
:1041B0005ECFCDB7DEB7E8E00C94302E81E080937F
:1041C000690580916905882349F080EE95E00E9499
:1041D000712B892BB1F30E942520F3CF0895AAE219
:1041E000B0E0E5EFF0E20C94122E0E9465286B011E
:1041F0007C0181E00E947E0A80EE95E00E94712B96
:10420000892B29F080EE95E00E949E2BF5CF2D980A
:1042100011E072E6B72EE9E2AE2E03E00E946528B7
:104220006C197D098E099F09693C7105810591050D
:10423000D0F11123C1F10E9465286B017C012C9AF9
:1042400080ED97E00E94A807B982E4E7F5E0DE017F
:1042500012968A2D01900D928A95E1F76AE2CE01BD
:1042600001960E94DB0B2C9880E090E00E94A8074A
:10427000009371050E94590B62E370E080E090E0CA
:104280000E94942880917105843061F40093710537
:104290008FE70E9477090E948A0911E0823419F49D
:1042A00010E001C011E08BE00E948A29892B81F483
:1042B00011E00EC02D9A2C9A80EE95E00E949E2B64
:1042C0008D309105A9F05CF40A9791F02D982C9807
:1042D00080EE95E00E94712B892B61F79FCF83328E
:1042E000910579F08234910589F70E94DE20EECFA6
:1042F00062EB71E080EE95E00E944B2A0E94471D20
:10430000E5CF0E94D215E2CF8F929F92AF92BF92DB
:10431000CF92DF92EF92FF921F93CF93DF938BE0C8
:104320000E948A29892B09F089C068EC70E080E03E
:1043300090E00E94942880E090E00E94A8070E94EC
:1043400065284B015C016B017C0180ECC80E82E1A9
:10435000D81EE11CF11C0E9465286C157D058E0598
:104360009F0530F48BE00E948A29892BA1F364C059
:104370008BE00E948A29892B09F05EC080ED97E0CE
:104380000E94A8070E9465286B017C01D0E0C1E073
:1043900088E4880E86E2981EA11CB11C11E08BE017
:1043A0000E948A29892B21F58C149D04AE04BF0438
:1043B00030F480ED97E00E94A807D1E0F0CF0E9492
:1043C00065286C197D098E099F09693C7105810575
:1043D000910528F30E9465286B017C01C12719F023
:1043E00080ED97E002C080E090E00E94A807D7CF60
:1043F00080E090E00E94A807DD23B9F08091D1050C
:1044000090E0019665E070E00E94B52D8093D105A3
:104410000E94290D0E94A9130E94480D64EF71E0CB
:1044200080E090E00E94942809C080E00E94DF06AE
:104430000E94C0110E943F0D0E94EF20DF91CF919A
:104440001F91FF90EF90DF90CF90BF90AF909F9023
:104450008F900895CF92DF92EF92FF9280E00E94BA
:10446000DA070E94B10761E08DE00E941E2961E039
:104470008CE00E941E2960E08BE00E941E2960E013
:1044800083E00E941E2961E083E00E94572961E0D9
:104490008EE00E941E2960E08EE00E9457290E9453
:1044A0009F0740E052EC61E070E080EE95E00E94F2
:1044B000B92C0E94A9130E94480D0E9492138FEFFD
:1044C0008093A8040E94C60778940E9465286B0117
:1044D0007C018091A8048F3F59F40E9465286C19D3
:1044E0007D098E099F09603D77408105910588F31C
:1044F00080ED97E00E94A80761E08BE00E945729B9
:104500002D9A80EE95E00E94712B892B29F080EE88
:1045100095E00E949E2BF5CF6DEF72E080EE95E066
:104520000E942C2A82E893E00E94300C64E173E040
:1045300080EE95E00E942C2A4AE050E062E070E0B4
:1045400080EE95E00E94FC2A62E370E080E090E05B
:104550000E94942880EE95E00E94712B04970CF144
:1045600080EE95E00E949E2B82349105D1F480EE7E
:1045700095E00E949E2B8E34910599F480EE95E093
:104580000E949E2B8434910561F480EE95E00E9498
:104590009E2B819731F480E090E00E94A8070E9452
:1045A000EF204091750550917605609177057091E7
:1045B0007805DB01CA010197A109B1090497A1059A
:1045C000B10568F44093A704433029F440EA56E863
:1045D00061E070E004C040E052EC61E070E080EE29
:1045E00095E00E94B92C0E9484212D9880E090E0F3
:1045F0000E94A8070E9492131092C3048091BD05E7
:1046000083FF11C080918905882351F08091900526
:10461000882331F080919705882311F087E001C04D
:1046200085E08093C30480E00E947E0A8091C404E8
:104630000E94B2090E94590B10923F0410923E044E
:1046400010923D04F12C8091D2058F15B0F062E3F9
:1046500070E080E090E00E94942880ED97E00E9456
:10466000A80762E370E080E090E00E94942880E078
:1046700090E00E94A807F394E6CF80919C0584FF08
:1046800008C0982F987181E0983109F080E00E946D
:104690007C118FE00E94DA07FF90EF90DF90CF90BF
:1046A0000895EF92FF920F931F93CF93DF938C01A6
:1046B0006EE770E080EE95E00E945906E801F12C6B
:1046C000F0E2EF2E8E0188818D57823048F46DE73D
:1046D00070E080EE95E00E94590688818E258883DF
:1046E0002196F801608180EE95E00E94CB2BF39437
:1046F000F9E0FF12E7CF6EE770E080EE95E00E94F0
:104700005906CDB7DEB7E6E00C94322EA9E0B0E052
:10471000ECE8F3E20C941A2E9091C50491110EC0AE
:104720009EEF99838A836B8350E0559547954C8320
:104730002D83198618861F821E822EC04091CA04BE
:10474000842F90E0B4E095958795BA95E1F7242FF2
:104750002F7030E08217930719F18DEF89831B8248
:10476000FE01349650E0842F90E0A4E09595879563
:10477000AA95E1F7242F2F7030E08217930749F0B4
:10478000DC01A553BB4F8C918193405F5F5F563036
:1047900051F74093CA045A83CE0101960E945123D7
:1047A0008091C50490E0019666E070E00E94B52D0E
:1047B0008093C5042996E2E00C94362EA0E0B0E088
:1047C000E4EEF3E20C94132E6C016EE770E080EEE1
:1047D00095E00E9459068601E12CF12CC0E0D0E062
:1047E00030E2B32EF801608183E8860F823078F4DE
:1047F0006DE770E080EE95E00E945906F801608157
:104800006B2570E080EE95E00E94590604C080EEB2
:1048100095E00E94CB2BE114F10459F0F80180815E
:104820009E01280F311DC901C92FDD27C80FD91FCF
:10483000DD273FEFE31AF30A89E0E816F10459F0A7
:1048400028E0E216F10421F48C2F8095F601808790
:104850000F5F1F4FC7CFCDB7DEB7E9E00C942F2E07
:10486000A9E0B0E0E6E3F4E20C941A2EE82F362F2C
:104870008091C50490E0019664E270E00E94B52D3D
:104880008093C50458E9598350E15A83813089F0F7
:1048900048F08230B9F08330D9F48B8381EF8C8378
:1048A0003D8319C085E08B8381EF8C832F5F2D833F
:1048B00012C08B8381EF8C8384E6489FA001112472
:1048C0005D8309C084E08B8381EF8C83ED8303C01B
:1048D0000E94B91104C0CE0101960E94DE232996E0
:1048E000E2E00C94362EA2E0B0E0E9E7F4E20C94AA
:1048F0000F2E182F762E2A8349830E9471286B0170
:104900007C018091DB048090C6049090C704A09045
:10491000C804B090C9042A8149818823C1F0D70115
:10492000C60188199909AA09BB094C015D0191EEDC
:1049300089169EE29906A104B10420F1241708F417
:10494000422F202F672D812F0E94302413C0D701C2
:10495000C60188199909AA09BB094C015D0191E3B7
:10496000891695E79906A104B10460F0672D812F9F
:104970000E948623C092C604D092C704E092C80465
:10498000F092C9042296EDE00C942B2EA2E2B0E046
:10499000ECECF4E20C94102E8CE00E949909811149
:1049A0000DC06CE173E080EE95E00E945D2A2D9AC7
:1049B00080E00E947E0A0E94590B2D9880EE95E0BF
:1049C0000E94712B892B01F180EE95E00E949E2BB5
:1049D0009091A704992319F00E94BC13EFCF409146
:1049E0003E0450E09A012F5F3F4F2F7133276091B3
:1049F0003F0470E02617370709F3FA01E75BFB4F26
:104A0000808320933E04DACF80917105843009F0D1
:104A100086C00E947128611571058105910549F0D4
:104A20006093B5047093B6048093B7049093B80470
:104A30000CC081E090E0A0E0B0E08093B5049093DA
:104A4000B604A093B704B093B8048091AB049091DE
:104A5000AC0481609093AC048093AB0483E08093BA
:104A600071058FE70E94770909E614E00E948A0920
:104A7000F80181938F01F4E002371F07B9F7209105
:104A8000720480916904982F922796FF3BC090E4AE
:104A9000922790937204982F98739833F1F410E052
:104AA000212F30E080916904877090E0821793078E
:104AB0004CF11F5F20919C05812F90E0FC01E7598C
:104AC000FB4F24FF04C080810E949B11E9CF6081CD
:104AD00080EE95E00E94CB2BE3CF8F7399F4809109
:104AE0006A048093B40480916B048093B204809133
:104AF0006C048093B10480916F0490E09093AA04B9
:104B00008093A90480913D04813019F482E0809360
:104B10003D0480913D04833011F410923D040E94C5
:104B200071286B017C018091AD049091AE04A0913D
:104B3000AF04B091B0040097A105B105C9F0A70179
:104B40009601281B390B4A0B5B0BDA01C901883B24
:104B50009B40A105B10560F00E94C8098093B30491
:104B60001092AD041092AE041092AF041092B004F3
:104B70008091B9049091BA04A091BB04B091BC0497
:104B800046015701881A990AAA0ABB0A84E795E0E8
:104B90000E94F40786169706A806B90608F4A8C06E
:104BA000C092B904D092BA04E092BB04F092BC0463
:104BB0000E9457068091A8048830A0F08091BD051E
:104BC0009091BE05A091BF05B091C0055CE1B6957E
:104BD000A795979587955A95D1F7892B8A2B8B2B7B
:104BE00009F09EC18091A8048F5F8093A8048091F2
:104BF000B5049091B604A091B704B091B8040097A1
:104C0000A105B105F1F0C81AD90AEA0AFB0A84E73E
:104C100095E00E94F4076C157D058E059F0508F050
:104C200006C18091BD0584FD04C080ED97E00E941F
:104C3000A8071092B5041092B6041092B70410920F
:104C4000B80490917204907C9093720450913E0449
:104C500080913F0420913D04581709F405C122308A
:104C600009F002C1905890937204E0919C05E7709E
:104C7000F0E0E658FC4F6081693008F0DDC061501B
:104C800040E04613DBC080933F0487E3840F90919C
:104C90007204892B809372044093400483E08093D4
:104CA0003D042C9A809181059091C304911129C1F2
:104CB0000E94790A8091C4040E94B209E0919C0587
:104CC000E770F0E0E658FC4F608182E794E00E94D4
:104CD000940BE091C404EF5FE093C404E83109F45D
:104CE0001CC1F0E0EC58FA4F8785882309F415C100
:104CF0000E94030C813069F580919C05887149F10F
:104D00008091AB049091AC04880F991F9093AC04F0
:104D10008093AB0483E0809371050E94590B0E943D
:104D200071286093AD047093AE048093AF049093A8
:104D3000B004672B682B692B61F481E090E0A0E060
:104D4000B0E08093AD049093AE04A093AF04B09311
:104D5000B00480919C0584FF1FC08091AB049091AA
:104D6000AC048E7F0E942A09182F6091A9048091BB
:104D7000B4040E94B213482F612F8091B30449A359
:104D80000E94B2130091D205282F49A16091B1046D
:104D90008091B2040E9473242C988091C1048130C8
:104DA000C1F018F08230B1F1C8C08BE00E948A29AE
:104DB000892B09F0C2C081E08093C1040E9465285C
:104DC0006093BD047093BE048093BF049093C004AD
:104DD000B4C08BE00E948A29892B31F50E94652896
:104DE000C090BD04D090BE04E090BF04F090C00419
:104DF0006C197D098E099F09693E734081059105F3
:104E000008F49BC082E08093C10480ED97E00E948B
:104E1000A80793C08BE00E948A29892B09F48DC0D2
:104E200080E090E00E94A8071092C10486C080E054
:104E300090E00E94A80705CF68E022CF851709F40B
:104E400022CF4F5F242F30E090E0F901EE58FB4F66
:104E5000DC01A75BBB4F7C917083F901E05CFB4FE9
:104E6000708301968F710DCF2430B1F420914004EE
:104E700081E494E0A3E7B4E0FC013E2F381B321735
:104E800018F431913D93F9CF87E3820F909172042A
:104E9000892B8093720402CF8091C104823051F437
:104EA0009160909372042D9A8E010F5F1F4FF12C29
:104EB000B80110C02D9880913D04811103C081E09C
:104EC00080933D0480913D04833071F784E08093AA
:104ED0003D04EACF8F2D69A37AA30E94B415F8018F
:104EE000819391938F01F39469A17AA1F0E1FF126C
:104EF000F1CF80919C0543E754E087700E947908C8
:104F0000D0CE882309F4D4CE2091C20431E0320FF0
:104F10003093C2042913CCCE0CC01092C404E8CE46
:104F20008091A804883009F42D9A89E08093A80420
:104F3000DFCE1092C2048150BBCEA296ECE00C945E
:104F40002C2E8230E8F4E82FF0E0EE0FFF1FED5238
:104F5000FA4F71836083813041F0809169008C7FCA
:104F6000842B80936900E89A089580916900440F2A
:104F7000551F440F551F837F842B80936900E99A46
:104F800008951F920F920FB60F9211242F933F9303
:104F90004F935F936F937F938F939F93AF93BF9341
:104FA000EF93FF938091D3059091D405892B29F03D
:104FB000E091D305F091D4050995FF91EF91BF9150
:104FC000AF919F918F917F916F915F914F913F91A1
:104FD0002F910F900FBE0F901F9018951F920F9258
:104FE0000FB60F9211242F933F934F935F936F93BC
:104FF0007F938F939F93AF93BF93EF93FF93809192
:10500000D5059091D605892B29F0E091D505F09131
:10501000D6050995FF91EF91BF91AF919F918F9127
:105020007F916F915F914F913F912F910F900FBEA4
:105030000F901F9018951F920F920FB60F92112488
:105040002F933F938F939F93AF93BF938091D805F6
:105050009091D905A091DA05B091DB053091D70583
:1050600023E0230F2D3720F40196A11DB11D05C0AB
:1050700026E8230F0296A11DB11D2093D70580932A
:10508000D8059093D905A093DA05B093DB058091FC
:10509000DC059091DD05A091DE05B091DF0501965C
:1050A000A11DB11D8093DC059093DD05A093DE0565
:1050B000B093DF05BF91AF919F918F913F912F9159
:1050C0000F900FBE0F901F9018952FB7F894609116
:1050D000D8057091D9058091DA059091DB052FBF35
:1050E00008953FB7F8948091DC059091DD05A0917B
:1050F000DE05B091DF0526B5A89B05C02F3F19F04E
:105100000196A11DB11D3FBF6627782F892F9A2FC9
:10511000620F711D811D911D42E0660F771F881F70
:10512000991F4A95D1F70895CF92DF92EF92FF929F
:10513000CF93DF936B017C010E947128EB01C114B6
:10514000D104E104F10479F00E9471286C1B7D0BFD
:10515000683E7340A0F381E0C81AD108E108F10865
:10516000C851DC4FECCFDF91CF91FF90EF90DF90F3
:10517000CF900895789484B5826084BD84B58160B1
:1051800084BD85B5826085BD85B5816085BDEEE64F
:10519000F0E0808181608083E1E8F0E0108280812E
:1051A00082608083808181608083E0E8F0E080819C
:1051B00081608083E1EBF0E0808184608083E0EBBC
:1051C000F0E0808181608083EAE7F0E080818460A4
:1051D0008083808182608083808181608083808100
:1051E000806880831092C1000895833081F028F494
:1051F000813099F08230A1F008958630A9F087308F
:10520000B9F08430D1F4809180008F7D03C080910B
:1052100080008F7780938000089584B58F7702C0D7
:1052200084B58F7D84BD08958091B0008F7703C0D1
:105230008091B0008F7D8093B0000895CF93DF936D
:1052400090E0FC01ED50F44F2491FC01E95FF34F35
:105250008491882349F190E0880F991FFC01E15D5A
:10526000F34FA591B4918B5D934FFC01C591D491FF
:105270009FB7611108C0F8948C91209582238C937C
:10528000888182230AC0623051F4F8948C91322FC5
:10529000309583238C938881822B888304C0F89473
:1052A0008C91822B8C939FBFDF91CF910895A1E0C9
:1052B000B0E0EDE5F9E20C94182E282F30E0F9016A
:1052C000E152F44F8491F901ED50F44F1491F9013A
:1052D000E95FF34F04910023C9F0882321F069832B
:1052E0000E94F5286981E02FF0E0EE0FFF1FEB5DD3
:1052F000F34FA591B4919FB7F8948C91611103C0BD
:105300001095812301C0812B8C939FBF2196E4E0EF
:105310000C94342ECF93DF93282F30E0F901E15223
:10532000F44F8491F901ED50F44FD491F901E95F04
:10533000F34FC491CC2391F081110E94F528EC2FFA
:10534000F0E0EE0FFF1FE55EF34FA591B4912C91B5
:105350002D2381E090E021F480E002C080E090E025
:10536000DF91CF9108958E3008F08E508770209194
:105370009D0190E4299F90011124822B80937C0051
:1053800080917A00806480937A0080917A0086FD13
:10539000FCCF809178002091790090E0922B0895C5
:1053A000A0E0B0E0E6EDF9E20C94142E6C017A0175
:1053B000EB01E60EF71E00E010E0CE15DF0561F010
:1053C0006991D601ED91FC910190F081E02DC6012B
:1053D0000995080F191FF1CFC801CDB7DEB7E8E076
:1053E0000C94302E6115710589F0DB010D900020C1
:1053F000E9F7AD0141505109461B570BDC01ED9116
:10540000FC910280F381E02D0995089580E090E001
:105410000895EF92FF920F931F93CF93DF938C0128
:10542000FB01C0E0D0E064917F018FEFE81AF80A39
:10543000662361F0D801ED91FC910190F081E02D9F
:10544000C8010995C80FD91FF701EDCFCE01CDB71F
:10545000DEB7E6E00C94322E0E94F2290895DC01BA
:10546000ED91FC910190F081E02D099508950F9345
:105470001F93CF93DF93EC016DE00E942F2A8C01E4
:105480006AE0CE010E942F2A800F911FDF91CF91F9
:105490001F910F9108950F931F93CF93DF93EC010A
:1054A0000E94092A8C01CE010E94372A800F911F89
:1054B000DF91CF911F910F9108950F931F93CF9379
:1054C000DF93EC010E94F2298C01CE010E94372A61
:1054D000800F911FDF91CF911F910F9108950F932E
:1054E0001F93CF93DF93EC010E942F2A8C01CE01F2
:1054F0000E94372A800F911FDF91CF911F910F914A
:105500000895A1E2B0E0E7E8FAE20C94102E7C01E5
:10551000C42EE52FCB01D22E19A221E02D1510F0BB
:105520002AE0D22E8E010F5D1F4F8D2C912CA12CC5
:10553000B12C6C2D7E2FA50194010E94C92D8C2DBC
:10554000D29E80191124015011098A3010F4805D17
:1055500001C0895CF80180832115310541055105A1
:1055600021F0C22EE32FCA01E4CFB801C7010E9487
:10557000F229A196ECE00C942C2EA0E0B0E0E3EC34
:10558000FAE20C94142EEC016A017B01211531051D
:1055900041F4E881F9810190F081E02D642F0995B3
:1055A0001DC02A303105A9F477FF12C06DE20E94B8
:1055B0002F2A8C0144275527BA014C195D096E0921
:1055C0007F092AE0CE010E94812A800F911F06C028
:1055D0002AE0B701A601CE010E94812ACDB7DEB72D
:1055E000E8E00C94302E9A01AB01662757FD6095D8
:1055F000762F0E94BD2A08950F931F93CF93DF93B8
:10560000EC019A01AB01662757FD6095762F0E9449
:10561000BD2A8C01CE010E94372A800F911FDF9195
:10562000CF911F910F9108952115310549F4DC01A7
:10563000ED91FC910190F081E02D642F0995089582
:105640000E94812A08959A01462F50E060E070E0A0
:105650000E94142B08959A01AB0160E070E00E9453
:10566000142B08950F931F93CF93DF93EC010E94A7
:10567000142B8C01CE010E94372A800F911FDF91DD
:10568000CF911F910F9108950F931F93CF93DF93A5
:10569000EC019A01AB0160E070E00E94142B8C01D8
:1056A000CE010E94372A800F911FDF91CF911F9169
:1056B0000F9108950F931F93CF93DF93EC019A01FD
:1056C000462F50E060E070E00E94142B8C01CE0168
:1056D0000E94372A800F911FDF91CF911F910F9168
:1056E0000895FC0124853585F901E05CFF4F808138
:1056F0009181F901EE5BFF4F20813181821B930B79
:105700008F7399270895FC0184859585FC01E05CE1
:10571000FF4F40815181FC01EE5BFF4F20813181C1
:105720004217530741F00190F081E02DE80FF91F77
:10573000808190E008958FEF9FEF0895FC018485AC
:105740009585FC01E05CFF4F40815181FC01EE5BDF
:10575000FF4F208131814217530779F0A081B18139
:10576000A80FB91F8C91208131812F5F3F4F2F737C
:1057700033273183208390E008958FEF9FEF0895C2
:10578000FC0181A1882329F0A489B5898C9186FF29
:10579000FBCF11A20895CF93DF93FC0126853785B7
:1057A000D901A05CBF4F8D919C91119701968F7389
:1057B0009927E901CE5BDF4F48815981841795070E
:1057C000D9F30D90BC91A02DA20FB31F6C93A685A9
:1057D000B785A05CBF4F11969C938E93A689B7891D
:1057E0002C9181E090E0078C02C0880F991F0A94E9
:1057F000E2F7282B2C9381E081A30488F589E02D22
:1058000080818064808381E090E0DF91CF91089572
:1058100008951F920F920FB60F9211242F933F936A
:105820004F938F939F93EF93FF938091C00082FDDE
:105830001CC04091C6008091860690918706019613
:105840008F739927209188063091890682179307D4
:1058500071F0E0918606F0918706EA5BF94F40838C
:10586000909387068093860602C08091C600FF91C0
:10587000EF919F918F914F913F912F910F900FBE7C
:105880000F901F90189580EE95E00E94712B892B48
:1058900011F00E94082C08951F920F920FB60F92DC
:1058A00011242F933F938F939F93EF93FF93209116
:1058B0004206309143068091440690914506281790
:1058C000390731F48091C1008F7D8093C10014C0ED
:1058D000E0914406F0914506EE5FF94F20818091FA
:1058E00044069091450601968F739927909345063B
:1058F000809344062093C600FF91EF919F918F9172
:105900003F912F910F900FBE0F901F901895A0E020
:10591000B0E0EDE8FCE20C94102EFC011382128240
:1059200088EE93E0A0E0B0E084839583A683B783FC
:105930008CEB93E0918380837587648757874687D4
:10594000318B208B138B028BF58AE48AD78AC68A27
:10595000B18EA08E938E828E8F85848F8889858F5D
:105960008989868F8A89878F8B8980A3ECE00C9444
:105970002C2ECF92DF92EF92FF92CF93DF93EC0128
:105980006A017B01411581EE580761057105F9F047
:10599000EC89FD8981E090E008A002C0880F991F82
:1059A0000A94E2F7808360E079E08DE390E0A7015C
:1059B00096010E94C92D215031094109510956957E
:1059C000479537952795211580E1380798F0EC89A0
:1059D000FD89108260E874E88EE190E0A7019601ED
:1059E0000E94C92D21503109410951095695479509
:1059F00037952795E889F9893083EA89FB892083DF
:105A000019A2EE89FF89408181E090E09C010C8C15
:105A100002C0220F331F0A94E2F7422B4083EE8923
:105A2000FF8940819C010D8C02C0220F331F0A9414
:105A3000E2F7422B4083EE89FF8940819C010E8C66
:105A400002C0220F331F0A94E2F7422B4083EE89F3
:105A5000FF8920810F8C02C0880F991F0A94E2F7FA
:105A6000809582238083DF91CF91FF90EF90DF902C
:105A7000CF9008958F929F92AF92BF92CF92DF9274
:105A8000EF92FF920F931F9381E08F9385E08F93A6
:105A900087E08F9383E08F9384E08F93E6EC8E2EE4
:105AA000912CF2ECAF2EB12CA1ECCA2ED12CB0EC83
:105AB000EB2EF12C04EC10E025EC30E042E056E057
:105AC00066E476E080EE95E00E94872C0F900F90C0
:105AD0000F900F900F901F910F91FF90EF90DF901C
:105AE000CF90BF90AF909F908F9008950E94BA285A
:105AF0000E942A22C3E4DCE20E94C6242097E1F33C
:105B00000E94432CF9CFA29FB001B39FC001A39F75
:105B1000700D811D1124911DB29F700D811D1124E6
:105B2000911D08950E94832DA59F900DB49F900D07
:105B3000A49F800D911D11240895B7FF0C94922D00
:105B40000E94922D821B930B0895DB018F939F93EC
:105B50000E94922DBF91AF91A29F800D911DA39F96
:105B6000900DB29F900D1124089597FB072E16F407
:105B7000009407D077FD09D00E94472E07FC05D07E
:105B80003EF4909581959F4F0895709561957F4F54
:105B90000895A1E21A2EAA1BBB1BFD010DC0AA1F6E
:105BA000BB1FEE1FFF1FA217B307E407F50720F086
:105BB000A21BB30BE40BF50B661F771F881F991F01
:105BC0001A9469F760957095809590959B01AC014A
:105BD000BD01CF010895052E97FB1EF400940E948D
:105BE000022E57FD07D00E94C92D07FC03D04EF4AA
:105BF0000C94022E50954095309521953F4F4F4F74
:105C00005F4F089590958095709561957F4F8F4F68
:105C10009F4F08952F923F924F925F926F927F9283
:105C20008F929F92AF92BF92CF92DF92EF92FF92AC
:105C30000F931F93CF93DF93CDB7DEB7CA1BDB0B58
:105C40000FB6F894DEBF0FBECDBF09942A883988FD
:105C500048885F846E847D848C849B84AA84B98404
:105C6000C884DF80EE80FD800C811B81AA81B98110
:105C7000CE0FD11D0FB6F894DEBF0FBECDBFED0124
:105C80000895EE0FFF1F0590F491E02D0994AA1BD3
:105C9000BB1B51E107C0AA1FBB1FA617B70710F017
:105CA000A61BB70B881F991F5A95A9F78095909549
:105CB000BC01CD0108958F929F92AF92BF92CF9277
:105CC000DF92EF92FF92CF93DF93EC0168817981AD
:105CD0008A819B81611571058105910521F464E23A
:105CE00079ED8BE597E02DE133EF41E050E00E9444
:105CF000EB2D49015A019B01AC01A7EAB1E40E94D6
:105D0000922D6B017C01ACEEB4EFA50194010E94D1
:105D1000A02DC60ED71EE81EF91EF7FE06C081E0B4
:105D2000C81AD108E10880E8F80AC882D982EA8254
:105D3000FB82C701B6019F77DF91CF91FF90EF9073
:105D4000DF90CF90BF90AF909F908F9008950E946A
:105D50005B2E089586E091E00E945B2E089560938B
:105D6000060170930701809308019093090108953B
:105D70002F923F925F926F927F928F929F92AF92FB
:105D8000BF92CF92DF92EF92FF920F931F93CF9328
:105D9000DF938B01EA016115710521F0DB018C9322
:105DA00011969C93209739F09E012250310923329D
:105DB000310508F0D8C07C016701BFEFCB1ADB0AC0
:105DC0005601F7016080862D90E00E94EA2F892B12
:105DD00011F07601F1CFFDE26F120AC0570182E0A7
:105DE000A80EB11CD70111966C90772473940BC048
:105DF000BBE26B1207C05701E2E0AE0EB11CD70147
:105E000011966C90712CCE018F7E892B89F4B0E3B2
:105E10006B1237C0F50180818F7D8835D1F46180A8
:105E2000F2E0AF0EB11C872D8260782EC0E1D0E089
:105E3000CA30D10551F1C031D10521F0C830D105AA
:105E400099F409C0CC24CA94DC2CEC2CAFE0FA2ED7
:105E500022C0209769F7C8E0D0E0CC24CA94DC2C9B
:105E6000EC2CFFE1FF2E17C06FEF7FEFCB019E01FF
:105E7000442737FD4095542F0E94C92D69017A01AE
:105E80000AC02097A9F6CAE0D0E0E9E9CE2EDC2CC2
:105E9000EC2CE9E1FE2EF50160E020E030E0A90104
:105EA0004E01AA2497FCA094BA2C1F0170ED572E26
:105EB000560CA9E0A51570F48FEB860D8A3118F405
:105EC00099EC592E06C08FE9860D8A3148F589EA8A
:105ED000582E560C852D90E08C179D070CF56F3FC2
:105EE000D9F0C216D306E406F50698F0C501B40150
:105EF0000E94A52D9B01AC01852D90E0A0E0B0E0B3
:105F0000280F391F4A1F5B1F281739074A075B07ED
:105F100010F46FEF01C061E03196D1016C90C5CFF4
:105F20000115110551F0662311F0319703C071FE80
:105F300004C03297D801ED93FC9370FE07C05095D2
:105F40004095309521953F4F4F4F5F4F67FF10C0F1
:105F500082E290E090938B0680938A066FEF7FEF4A
:105F60008FEF9FEF07C060E070E080E090E002C03C
:105F7000B901CA01DF91CF911F910F91FF90EF906E
:105F8000DF90CF90BF90AF909F908F907F906F9059
:105F90005F903F902F900895FC0188279927E894FF
:105FA00021912032E9F3293010F02E30C8F32B3242
:105FB00041F02D3239F4689404C00E941E30820FE3
:105FC000911D219120532A30C0F31EF490958195A4
:105FD0009F4F0895911150C0803219F0895085501B
:105FE000D0F7089548EC53E00E94F72F0895FA0186
:105FF000A191B081009719F41097E1F0CD01DC0177
:10600000CD010D90002011F4C00113C0FB012191BE
:10601000222319F02015D9F7F3CFFB012191201588
:1060200019F41E92119606C02223C1F70D9000208C
:10603000A1F7D001FA01A193B08308957AE0979F68
:10604000902D879F802D910D11240895F999FECFF1
:1060500092BD81BDF89A992780B50895262FF999A8
:10606000FECF1FBA92BD81BD20BD0FB6F894FA9A3B
:10607000F99A0FBE01960895992788270895F894F4
:02608000FFCF50
:1060820000008C06200001000000FF000200020058
:1060920002000200020002000200020002000200EE
:1060A2000200020002000200020002802500000538
:1060B200400AA1204EA50020244EA52C2330C01258
:1060C20000001A400AA1204EA5001B1E27522C23B5
:1060D200308025000005400AA1204EA50020244E54
:1060E200A52C2330004B000006400AD0009D490039
:1060F2007B289D492C233000E1000005400A450120
:10610200D7DC03B81E0EBF00232E48E801008A40E8
:106112000A6001555502AD1E20000023C8015458E3
:106122002074696D656F75742100596573004E6F37
:10613200002C00386368004E2F41002C205B005D6C
:106142002028002900486F70206368616E6E656CBC
:10615200200020402000456E746572696E672061E0
:1061620064617074697665206368616E6E656C2027
:1061720073656C656374696F6E2C207069636B69FB
:106182006E673A007363616E6E6572206D6F64654F
:10619200004E4F5420454E41424C45440053656EDB
:1061A20064696E672073657474696E677320746FB7
:1061B2002052580A00526573657474696E672073C1
:1061C200657474696E6773206F6E2052580A0041BD
:1061D200626F727465642065646974730A00696E23
:1061E20076616C69642073656C656374696F6E00B7
:1061F2000D0A496E76616C696420696E707574204F
:106202002D206469736361726465642107005365BC
:106212007474696E677320736176656420746F208D
:10622200454550524F4D0A00526576657274656459
:106232002073657474696E67732066726F6D204592
:106242004550524F4D0A004C6F616465642066618F
:1062520063746F72792064656661756C74730A0089
:106262004B657920616E64206368616E6E656C7344
:106272002072616E646F6D697A65640A004F7065A1
:106282006E4C52536E672054582073746172746955
:106292006E672000206F6E20485720006D6F647576
:1062A2006C65206C6F636B65643F00342B3400387F
:1062B20000382B340031320031322B3400313600B9
:1062C20050504D0052535349005344410053434CE4
:1062D20000525844005458440041494E004C424533
:1062E20045500053504B54524D00534255530053A6
:1062F200554D44004C4C494E440000070B0C101104
:106302001500B7012B032F033103350338033D0377
:10631200B7014003440349034D0351035503590395
:106322005D0363036A036F0374038D028D028D02A2
:106332008D02160A1322312900000000CB2BD0292E
:08634200712B9E2B832BC02B55
:107E00000F92CDB7DEB7112484B714BE81FFF1D035
:107E100082E08093C00088E18093C10086E0809377
:107E2000C20080E18093C4008EE0CDD088249924E4
:107E3000CC24C394F5E0DF2EE1E1EE2E73E0F72EC3
:107E4000B6D0082F813479F4B2D08983C2D0898129
:107E5000823811F481E005C0813811F485E001C059
:107E600083E09ED09AC0823411F484E103C085344B
:107E700019F485E0B6D091C0853561F498D0082F0B
:107E800010E095D090E0982E8824802A912A880CC2
:107E9000991C82C0863521F484E0A3D080E0E1CF34
:107EA000843609F04CC083D082D0A82E80D0B82E62
:107EB00000E011E07CD0F80181938F01AE16D1F77C
:107EC00088D0FB2DF53489F4E0E0F1E00BC0F9999E
:107ED000FECF92BC81BC0894811C911C819180BD15
:107EE000FA9AF99AEA1598F358C08B2D863409F05E
:107EF00054C0F401F7BEE89507B600FCFDCFF401CD
:107F0000A0E0B1E02C9130E011968C91119790E0B7
:107F1000982F8827822B932B12960C01C7BEE895C9
:107F20001124329681E0A038B80761F7F401D7BE7A
:107F3000E89507B600FCFDCFE7BEE8952EC0843774
:107F4000F1F435D034D0182F32D0B82E42D0FB2DDA
:107F5000F63421F4F40105914F010CC0FB2DF534EA
:107F600049F4F999FECF92BC81BC0894811C911C04
:107F7000F89A00B5802F14D0115049F70EC08537FC
:107F800039F427D08EE10CD085E90AD08FE069CF93
:107F9000813511F488E017D01CD080E101D050CF9A
:107FA0009091C00095FFFCCF8093C600089580910A
:107FB000C00087FFFCCF8091C00084FD01C0A89560
:107FC0008091C6000895E0E6F0E098E19083808318
:107FD0000895EDDF803219F088E0F5DFFFCF84E10E
:107FE000DFCF1F93182FE3DF1150E9F7F2DF1F9166
:0E7FF0000895282E80E0E7DFEE27FF27099492
:027FFE0001057B
:0400000300007E007B
:00000001FF
